:020000040000FA
:1000000086018501A9018F28F000030E8312A0004C
:100010000B1D0F28B308031DB3030B115028031049
:10002000A60DA50DA40DA30D051A2617A9182528A0
:100030005D212208D83A031D4F282108033A031DE9
:100040004F28A914A7010130A8005520A80B4F285C
:1000500002302706031D2F28D430AC193128270879
:100060007320A5065D2123308400402141211F30EB
:10007000220503193D28A9104F280310270D2A3EF9
:10008000840023088000840A240880001A30A80015
:10009000A70A271D4F282915A701F030B9008B109A
:1000A000200E8300F00E700E090039080F39031D71
:1000B0006B283908F039803A031972281A30B907C9
:1000C000FF30B91B6828390E0F392A3E840000081A
:1000D000BA00851472283A1885103A1C8514031446
:1000E000BA0CB903080082073F3466345A346D34C1
:1000F0008207A834A8348C34863481342D342034DB
:100100005034493443342D3452344434533420343D
:1001100032342E343034303420342D34FF34073030
:100120009F0083164730810011308500F130860032
:10013000831232302D220C228B1344220A22A30177
:10014000A401A501A601B401B2017F30B300B03013
:100150008B006400330803199C280739031DB42859
:10016000B3035522B20AB213291DA92829117030F0
:10017000B3042A082B0634060319C128A916B406AD
:10018000A928A91EC628A9124422B2012C08F039B8
:100190000319D328203A031912292C08F839403AB8
:1001A00003192229A9288F30F22120302C1DDB28A9
:1001B0002D302D1A2A30F3212C1DE1282D1A05157A
:1001C0002D1E05112D0D0639063A0319F328063A9E
:1001D0003B3E8B138400300880388000840A31084D
:1001E00080008B17A928BB1FA928BD1FA928BF1FE6
:1001F000A928BB13BC13BD13BE13BF13C01380309B
:10020000F2213B08F0213C08F0213D08F0213E0896
:10021000F0213F08F0214008F0213008F02131089A
:10022000F021A9282D0D3E39B600B6073208B602D6
:10023000B6132E08E3212F08E3213008E32131080B
:10024000E321A9288930F221300E0F392F181038F8
:10025000B500310C0F39B11A003CB5071830B51B89
:10026000B5073502031C350887223A30F321310DDA
:10027000B500300DB600350D360D3F398722A9285F
:1002800029148030A800A11C4C291F302205031D11
:100290004C292910280880060310A20DA10D291C45
:1002A0005729211D5729B930A2060130A106031094
:1002B000A80C031C4329840A0800A201A101261FDF
:1002C00065290330A1061B30A206A61F6B29033047
:1002D000A1068F30A206251C71290230A106A73085
:1002E000A206F730A518A206251D7A290130A1061D
:1002F000EE30A206A51D80290330A106DC30A2063F
:10030000251E86290230A1060130A206A51E8C29D1
:100310000130A106BB30A206251F92290330A10699
:100320007630A206A51F98290330A1065530A206F3
:10033000241C9E290330A1061330A206A41CA42964
:100340000330A1069F30A206241DAA290230A1066F
:100350008730A206B730A419A206241EB3290130A3
:10036000A1066E30A206A41EB9290230A106DC3017
:10037000A2060130241BA2060230A41BA2060430F0
:100380002318A2060830A318A20610302319A206CB
:100390002030A319A2064030231AA2068030A31AE7
:1003A000A2060130231BA1060230A31BA1060800F0
:1003B0000430860086140000060D86108614861010
:1003C0000318DA290800B7003608361BEC29273C49
:1003D000C030031C68303607F221B60AB61337085E
:1003E0000023F329A915B500D82183160130860012
:1003F000831235080322350E0322A9118316F1302A
:10040000860083120800F039A91D0838860086147A
:100410008610080005301E2AA9153030032203304B
:100420002D223030032201302D22303003220130C2
:100430002D222030032201302D22B60136087820EB
:10044000FF3A03190800FF3AB500A915B51FA91115
:100450007F39B500F321B60A1E2AB700B80164003F
:10046000B80B2F2AB70B2E2A0800D8218615861420
:10047000000006088610F039B50086140000060E4C
:1004800086100F39350408000130F2214030B600E3
:10049000F2212030F321B60B492A2030BB00BC00EA
:1004A000BD00BE00BF00C00008000430F221403093
:1004B000B700F2213522B6003F30B8007E22C030AE
:1004C000B700F2213522B8007F30F2213808F3213D
:1004D0002730B8007E229030B700F2213522B800D4
:1004E000E730F2213808F3211730B8007E22A73018
:1004F000F2213608F3210630F2210800B70A370846
:10050000F2213522F321B80B7E2A64000800B501E0
:10051000F63EB50A0318882AFA3EB50E3507B6002E
:10052000360E932236080F39063E8318073E2A3EC0
:02053000F329AD
:10060000B500B51B082BE039031920343508080064
:100610008B1303308A000E238A01090035087F39C5
:1006200082076134613465346534693469346F3408
:100630006F3475347534EE3443345334E2346934F2
:1006400069346134E13465346534693469346F3454
:10065000EF347534F534EE34633473347134693403
:1006600069346134E03463342534473465346E349E
:100670009434F7344334ED3424347F345E347E34A0
:100680007634DF343134323433342B3449346E34FD
:10069000F534E4343F34FD34DF3420342034203466
:1006A00024344134413445344534493449344F3499
:1006B0004F34553455345234433453345A3444341B
:1006C0004C344134E13445344534493449344F34B1
:1006D000EF345534F5347234633473347A3464341B
:1006E0006C344134413445344534793459344F34D1
:1006F000303470346E345234433453345A34FA3410
:1007000064346134613465346534773479346F34FA
:10071000F23470346E347234633473347A34FA34AD
:02072000203483
:02400E00673E0B
:00000001FF
